:020000040800F2
:10A0000070CC002059A10008F1BE00080DB5000871
:10A0100069BE0008EDA2000895CF0008000000000E
:10A020000000000000000000000000006DCB0008F0
:10A03000D5A90008000000005DC70008ADCD0008EC
:10A04000B9A10008B9A1000869CF00086DC30008D4
:10A05000D5C3000885AA0008B9A1000859A90008BD
:10A06000B9A10008B9A10008B9A10008B9A1000868
:10A07000C9BF0008B9A1000821C30008B9A10008A0
:10A08000B9A10008B9A10008B9A10008B9A1000848
:10A09000B9A10008B9A10008B9A10008B9A1000838
:10A0A00091CF0008B9A10008B9A10008B9A1000822
:10A0B000B9A10008B9A10008B9A10008B9A1000818
:10A0C000B9A10008D1C70008B9A10008B9A10008CA
:10A0D000B9A100080DC4000815C400081DC400087B
:10A0E00025C40008CDAA0008E9AA0008B9A1000803
:10A0F00005AB0008B9A1000821AB00083DAB000882
:10A1000059AB000875AB00089DAB0008C5AB000853
:10A11000EDAB000815AC00083DAC000865AC0008CC
:10A120008DAC0008B9A10008B9A1000857B5000816
:10A130005FB50008F1C70008B9A10008B9A100087F
:10A14000DFF810D000F098F800480047FDD600086E
:10A15000AFF3008070CC0020184880474FF080405B
:10A160004FF04021C8654000C8654010C8650846EA
:10A17000C06D40F48000C86511484FF0402148652B
:10A180004FF04021C86D20F04040C8650D48804721
:10A190004FF00E000C494FF000000C4908800C48AD
:10A1A00080470C480047FEE7FEE7FEE7FEE7FEE7D4
:10A1B000FEE7FEE7FEE7FEE7FEE70000B9BD0008A8
:10A1C00000100081D9B70008005000400060004036
:10A1D000D9CE000841A100082DE9F05F0546002016
:10A1E00092469B4688460646814640241BE0284608
:10A1F00041464746224600F02FF853465A46C01AB9
:10A20000914110D311461846224600F016F82D1A37
:10A2100067EB01084F4622460120002100F00DF8AF
:10A2200017EB00094E41201EA4F10104DFDC484673
:10A2300031462A464346BDE8F09F202A04DB203AF7
:10A2400000FA02F1002070479140C2F1200320FA89
:10A2500003F3194390407047202A04DB203A21FA87
:10A2600002F00021704721FA02F3D040C2F120022F
:10A270009140084319467047064C074D06E0E068D8
:10A2800040F0010394E8070098471034AC42F6D33D
:10A29000FFF75AFF44DC000864DC000870B5044690
:10A2A0000D46E1B25A2001F0C5FB21125B2001F0FE
:10A2B000C1FBE9B25C2001F0BDFB29125D2001F079
:10A2C000B9FB70BD70B504460D46E1B2562001F0F1
:10A2D000B1FB2112572001F0ADFBE9B2582001F08B
:10A2E000A9FB2912592001F0A5FB70BD10B503A0F0
:10A2F00002F08CFE02F0C9FC10BD00007761726EA6
:10A30000696E67A3BB4275734661756C74204861C2
:10A310006E646C65720D0A004FF04021096A41F0CD
:10A3200001014FF04022116200BF4FF04021096A45
:10A3300001F48071B1F5807FF7D14FF04021496A77
:10A3400021F003014FF0402251621146496A5162E7
:10A3500000BF4FF04021496A01F48071B1F5807F60
:10A36000F7D15249524A1160032806D1111F0968DA
:10A3700041F08041121F116007E04D49091F096833
:10A3800021F080414A4A121F11604FF4C601484A29
:10A39000121D11604FF4B20111604FF40C111160E5
:10A3A0004FF4580111601160D1064FF04022D16581
:10A3B0004900D1654910D1655101D16560B93D4968
:10A3C000096801F07F41B1F1124F37D1394909686D
:10A3D00021F07F41916631E0022810D135490831E2
:10A3E000096801F07F41B1F1124F27D1314908319D
:10A3F000096821F07F414FF0402291661EE003285A
:10A400000CD12C49FC3109682B4A914216D12949BB
:10A41000F83109684FF0402291660FE02549091D87
:10A42000096801F07F41B1F1124F07D12149091D9F
:10A43000096821F07F414FF04022916600211C4ABB
:10A44000121D11601A49091F096821F08041184A3C
:10A45000121F116015493039121D11604FF0402153
:10A46000096A41F008014FF04022116200BF4FF02D
:10A470004021096A01F40061B1F5006FF7D14FF096
:10A480004021496A21F003014FF0402251621146F8
:10A49000496A41F00101516200BF4FF04021496A11
:10A4A00001F40071B1F5007FF7D170473099D8D829
:10A4B00004380040C00020083598746770B5024623
:10A4C0000B46274D2D6845F08045254E3560351DDE
:10A4D0002D78244E45EA0604224D3035204E361D97
:10A4E0003560214D2D6845F2AA56B5421DD14FF079
:10A4F0004025296B53B102F004051DB1114321F031
:10A5000004010DE0114381F0040109E002F00405AB
:10A510001DB1914341F0040102E0914381F0040137
:10A520004FF0402529635A2010E03BB14FF0402501
:10A530002D6B15434FF04026356306E04FF0402564
:10A540002D6B95434FF040263563FF20044D2D1DA4
:10A550002C602D1F2D6825F08045014E356070BDA3
:10A56000003800400099D8D8A400200870B50446EF
:10A570000D46072000F078FA34B1012C2AD0022CC5
:10A5800050D0032C76D176E04FF04020006A40F0A6
:10A5900001004FF04021086200BF4FF04020006AE8
:10A5A00000F48070B0F5807FF7D14FF04020406A12
:10A5B00020F003004FF0402148620846406A48629C
:10A5C00000BF4FF04020406A00F48070B0F5807FFB
:10A5D000F7D179E04FF04020006A40F008004FF0DA
:10A5E0004021086200BF4FF04020006A00F4006084
:10A5F000B0F5006FF7D14FF04020406A20F0030023
:10A600004FF0402148620846406A40F0010048622D
:10A6100000BF4FF04020406A00F40070B0F5007FAA
:10A62000F7D151E04FF04020006A40F004004FF0B5
:10A630004021086200BF4FF04020006A00F48060B3
:10A64000B0F5806FF7D14FF04020406A20F0030052
:10A650004FF0402148620846406A40F002004862DC
:10A6600000BF4FF04020406A00F48060B0F5806F7A
:10A67000F7D129E027E04FF04020006A40F01000B9
:10A680004FF04021086200BF4FF04020006A00F404
:10A690008050B0F5805FF7D14FF04020406A20F045
:10A6A00003004FF0402148620846406A40F0030032
:10A6B000486200BF4FF04020406A00F40060B0F5EF
:10A6C000006FF7D100E000BF00BF284602F00CFF8A
:10A6D00070BD00B5034600F01EF84FF04020C06D7D
:10A6E00040F400004FF04021C865102B05D108460A
:10A6F000006D40F4004008650CE04FF04020006D14
:10A7000020F400404FF0402108650846006D63F3D7
:10A710000300086500BD4FF04021C96D21F04040A5
:10A720004FF04021C86540F080414FF04022D16594
:10A7300040F00041D16540F04041D165704770B5AF
:10A7400002460B46002114461D46002002E0265C0E
:10A750003144401CA842FADB0846CE1701EB1666CE
:10A760003612A1EB0621C8B270BD10B50446E1B2A5
:10A77000502001F05FF9C4F30721512001F05AF98C
:10A78000C4F30741522001F055F9210E532001F086
:10A7900051F910BD10B50446E1B2542001F04AF958
:10A7A0002112552001F046F910BD10B500BF01F08F
:10A7B0004BF900F008000028F9D110BD10B500BF1A
:10A7C00001F042F900F008010029F9D110BD10B5DF
:10A7D00000BF01F039F900F004010029F9D010BDE3
:10A7E00030B530B9534C646A24F47F44514D6C62E7
:10A7F0001AE001280BD14F4C646A24F47F444D4D7C
:10A800006C622C46646A44F42A446C620CE00228B0
:10A810000AD1484C646A24F47F44464D6C622C464D
:10A82000646A44F47F446C6232B9424C246A24F472
:10A830004034404D2C621AE0012A0BD13D4C246A71
:10A8400024F440343B4D2C622C46246A44F40034FA
:10A850002C620CE0022A0AD1364C246A24F44034DB
:10A86000344D2C622C46246A44F440342C6233B9B3
:10A87000304C646A24F47F042E4D6C621AE0012B84
:10A880000BD12C4C646A24F47F042A4D6C622C4654
:10A89000646A44F42A046C620CE0022B0AD1254C51
:10A8A000646A24F47F04234D6C622C46646A44F489
:10A8B0007F046C6231B91F4C646A24F0FF041D4DA3
:10A8C0006C6222E001290FD11B4C1A4D80352C609F
:10A8D000184C646A24F0FF04164D6C622C46646ABE
:10A8E00044F0AA046C6210E002290ED1124C114D02
:10A8F00080352C600F4C646A24F0FF040D4D6C62AF
:10A900002C46646A44F0FF046C620A4C246844F0EC
:10A910000544084D2C6000BF064C246804F0004438
:10A92000B4F1004FF8D0034C246844F00104014D09
:10A930002C6030BD00500540FFFF1F0010B51320F4
:10A9400000F094FF00F0A3FFC4B204F0DF0420463F
:10A9500000F0B0FF10BD00001C480068806A1B4872
:10A960000068806C00F00F0060B118480068806CCF
:10A9700000F00F001649086008460068134909688E
:10A98000C1F8980011480068806A10490968886712
:10A990000E480068006B0D490968C1F880000B483B
:10A9A0000068806B09490968C1F888000748006899
:10A9B000006C06490968C1F8900004480068806C82
:10A9C00002490968C1F8980070470000E0000020C3
:10A9D000E800002010B503A002F018FB02F055F9C2
:10A9E00010BD00007761726E696E67A3BB4465623B
:10A9F00075674D6F6E2048616E646C65720D0A005C
:10AA000001B581B000200A49096841F27072B1FBBA
:10AA1000F2F1009105E000E0401C00998842FBD370
:10AA2000002001994A1E01920029F4D10CBD0000BA
:10AA3000C400002010B5CD2000F018FF00F027FF63
:10AA4000C4B204F07F04204600F034FF10BD10B5FE
:10AA5000122000F00BFF00F01AFFC4B244F04004D3
:10AA6000204600F027FF10BD0146054A106820F07F
:10AA70000F0001F00F021043014A10607047000000
:10AA8000003800400E48406800F0020040B101204C
:10AA90000C4908700A48406840F0020008494860C4
:10AAA0000748406C00F0020040B1012006490870E0
:10AAB0000348406C40F002000149486470470000C0
:10AAC00000A00040EC000020ED00002010B50021A7
:10AAD000034800F05FFA0021024800F05BFA10BD65
:10AAE000009001400040024010B50121034800F0F1
:10AAF00051FA0121024800F04DFA10BD00900140CA
:10AB00000040024010B50321034800F043FA03213E
:10AB1000024800F03FFA10BD0090014000400240A2
:10AB200010B50521034800F035FA0521024800F070
:10AB300031FA10BD009001400040024010B50621DE
:10AB4000034800F027FA0621024800F023FA10BD5E
:10AB5000009001400040024010B50721034800F07A
:10AB600019FA0721024800F015FA10BD00900140C3
:10AB70000040024010B50021054800F00BFA00210A
:10AB8000044800F007FA0021034800F003FA10BD62
:10AB900000A00140005002400060024010B50121B9
:10ABA000054800F0F7F90121044800F0F3F901210C
:10ABB000034800F0EFF910BD00A001400050024032
:10ABC0000060024010B50221054800F0E3F90221BF
:10ABD000044800F0DFF90221034800F0DBF910BD62
:10ABE00000A00140005002400060024010B5032167
:10ABF000054800F0CFF90321044800F0CBF9032108
:10AC0000034800F0C7F910BD00A001400050024009
:10AC10000060024010B50421054800F0BBF9042192
:10AC2000044800F0B7F90421034800F0B3F910BD5F
:10AC300000A00140005002400060024010B5052114
:10AC4000054800F0A7F90521044800F0A3F9052103
:10AC5000034800F09FF910BD00A0014000500240E1
:10AC60000060024010B50621054800F093F9062166
:10AC7000044800F08FF90621034800F08BF910BD5D
:10AC800000A00140005002400060024010B50721C2
:10AC9000054800F07FF90721044800F07BF90721FF
:10ACA000034800F077F910BD00A0014000500240B9
:10ACB0000060024070B504460D46002C4DD0012CBA
:10ACC0004BD0022C49D0032C47D0042C45D0052C66
:10ACD00043D0062C41D0072C3FD0082C3DD0092C66
:10ACE0003BD00A2C39D00B2C37D00C2C35D00D2C66
:10ACF00033D00E2C31D00F2C2FD0102C2DD0112C66
:10AD00002BD0122C29D0132C27D0142C25D0152C65
:10AD100023D0162C21D0172C1FD0182C1DD0192C65
:10AD20001BD01A2C19D01B2C17D01C2C15D01D2C65
:10AD300013D01E2C11D01F2C0FD0202C0DD0212C65
:10AD40000BD0222C09D0232C07D0242C05D0252C65
:10AD500003D0262C01D0272C00D103E0B02181A004
:10AD600002F0A0FB0DB1012D00D103E0B1217DA0C7
:10AD700002F098FB272C02DD4FF0FF3070BD092C4C
:10AD800009DB0B2C07DC4FF08040C06940F001006C
:10AD90004FF08041C8610E2C09DB0F2C07DC4FF00F
:10ADA0008040C06920F002004FF08041C861262C2D
:10ADB00009DB272C07DC4FF08040C06940F004001D
:10ADC0004FF08041C861062C09DB072C07DC4FF0EF
:10ADD0008040C06920F010004FF08041C861202CF5
:10ADE00009DB252C07DC4FF08040C06940F0800073
:10ADF0004FF08041C8611A2C09DB1F2C07DC4FF093
:10AE00008040C06940F480504FF08041C861162CEA
:10AE10000EDB192C0CDC4FF08040406C20F07040B1
:10AE20004FF0804148640846C06940F40050C86152
:10AE3000122C09DB152C07DC4FF08040C06940F470
:10AE400080404FF08041C861102C09DB112C07DCD9
:10AE50004FF08040C06940F400404FF08041C8612D
:10AE6000A5BBE01040B94648C07822460121914078
:10AE700088434349C87072E00120B0EBE40F09D168
:10AE80004048C078A4F1080101228A4090433D491E
:10AE9000C87064E00220B0EBE40F09D13A48C078F2
:10AEA000A4F1100101228A4090433749C87056E04E
:10AEB0000320B0EBE40F0AD13448C078A4F11801A4
:10AEC00001228A4090433149C87048E009E0304887
:10AED000C078A4F1200101228A4090432C49C87017
:10AEE0003DE0E01040B92648C0782246012191405B
:10AEF00008432349C87032E00120B0EBE40F09D1C8
:10AF00002048C078A4F1080101228A4010431D495D
:10AF1000C87024E00220B0EBE40F09D11A48C078D1
:10AF2000A4F1100101228A4010431749C87016E0AD
:10AF30000320B0EBE40F09D11448C078A4F1180144
:10AF400001228A4010431149C87008E01048C078B7
:10AF5000A4F1200101228A4010430D49C87000204D
:10AF60000CE700004D43555F6472765C6472765C5A
:10AF70007372635C65706F72745F6472762E6300C7
:10AF80000090014000A001400040024000500240FB
:10AF90000060024070B504460D46E67931461BA0BC
:10AFA00002F034F80120A840304000282CD0E0798D
:10AFB0000121A9400843E0712048844204D12A4677
:10AFC00000211FA002F022F82648844204D12A461C
:10AFD00001211BA002F01AF82348844204D12A461A
:10AFE000022117A002F012F82048844204D12A4618
:10AFF000032113A002F00AF81D48844204D12A4616
:10B0000004210FA002F002F870BD0000656E7465A7
:10B01000722065706F727420696E746572727570DB
:10B02000742E63757272656E7420737461747573B7
:10B03000203D20253032780D0A00000000900140AC
:10B04000456E7465722045504F5254256420696ED8
:10B05000746572727570742E50494E203D202564BF
:10B060000D0A000000A001400040024000500240D4
:10B070000060024070B504460D46002C4DD0012CF6
:10B080004BD0022C49D0032C47D0042C45D0052CA2
:10B0900043D0062C41D0072C3FD0082C3DD0092CA2
:10B0A0003BD00A2C39D00B2C37D00C2C35D00D2CA2
:10B0B00033D00E2C31D00F2C2FD0102C2DD0112CA2
:10B0C0002BD0122C29D0132C27D0142C25D0152CA2
:10B0D00023D0162C21D0172C1FD0182C1DD0192CA2
:10B0E0001BD01A2C19D01B2C17D01C2C15D01D2CA2
:10B0F00013D01E2C11D01F2C0FD0202C0DD0212CA2
:10B100000BD0222C09D0232C07D0242C05D0252CA1
:10B1100003D0262C01D0272C00D104E040F22311CB
:10B120005AA002F0BFF90DB1012D00D104E04FF497
:10B13000927156A002F0B6F9272C00DD70BDE01028
:10B14000D8B95948C0782246012191400843564950
:10B15000C870012D08D1084640792246012191404E
:10B160000843514948718FE04F48407922460121F8
:10B17000914088434C49487186E00120B0EBE40FD0
:10B180001ED14A48C078A4F1080101228A40104328
:10B190004649C870012D09D108464079A4F108013B
:10B1A00001228A401043414948716DE03F4840798F
:10B1B000A4F1080101228A4090433C49487163E0B0
:10B1C0000220B0EBE40F1ED13948C078A4F1100181
:10B1D00001228A4010433649C870012D09D1084622
:10B1E0004079A4F1100101228A401043304948718E
:10B1F0004AE02F484079A4F1100101228A4090438F
:10B200002B49487140E00320B0EBE40F1ED12948E0
:10B21000C078A4F1180101228A4010432549C87062
:10B22000012D09D108464079A4F1180101228A4074
:10B2300010432049487127E01E484079A4F11801C5
:10B2400001228A4090431B4948711DE01A48C0788A
:10B25000A4F1200101228A4010431749C870012D32
:10B2600009D108464079A4F1200101228A40104307
:10B270001149487108E010484079A4F120010122E9
:10B280008A4090430C49487100BF57E74D43555FD2
:10B290006472765C6472765C7372635C65706F7204
:10B2A000745F6472762E63000090014000A001403C
:10B2B00000400240005002400060024010B5CD2026
:10B2C00000F0D4FA00F0E3FAC4B244F0800420465F
:10B2D00000F0F0FA10BD10B5CD2000F0C7FA00F074
:10B2E000D6FAC4B204F0BF04204600F0E3FA10BD61
:10B2F00010B5CD2000F0BAFA00F0C9FAC4B244F09B
:10B300004004204600F0D6FA10BD10B5CD2000F064
:10B31000ADFA00F0BCFAC4B204F0FD0404F0FE047F
:10B32000204600F0C7FA10BD10B5CD2000F09EFAFF
:10B3300000F0ADFAC4B204F0FD0444F0010420466C
:10B3400000F0B8FA10BD10B5CD2000F08FFA00F073
:10B350009EFAC4B244F0020404F0FE04204600F059
:10B36000A9FA10BD10B5CD2000F080FA00F08FFAD8
:10B37000C4B244F0020444F00104204600F09AFAFA
:10B3800010BD10B5CC2000F071FA00F080FAC4B204
:10B3900004F0DF0444F01004204600F08BFA10BDE6
:10B3A00010B5CC2000F062FA00F071FAC4B244F09B
:10B3B000200404F0EF04204600F07CFA10BD10B524
:10B3C000CC2000F053FA00F062FAC4B204F0DF04BB
:10B3D00004F0EF04204600F06DFA10BD10B5CD204A
:10B3E00000F044FA00F053FAC4B204F0F70404F099
:10B3F000FB04204600F05EFA10BD10B5CD2000F031
:10B4000035FA00F044FAC4B204F0F70444F004043E
:10B41000204600F04FFA10BD10B5CD2000F026FAFE
:10B4200000F035FAC4B244F0080404F0FB042046EE
:10B4300000F040FA10BD10B5CD2000F017FA00F072
:10B4400026FAC4B244F0080444F00404204600F094
:10B4500031FA10BD4FF04020406A00F00302101E88
:10B4600006D0012806D0022817D0032819D116E0EB
:10B47000114918E01148006808B911490CE00F485B
:10B480000068012801D10F4906E00C480068022835
:10B4900001D10D4900E00D4905E00D4903E00D49DA
:10B4A00001E0002100BF00BF4FF040208068C0B223
:10B4B000401CB1FBF0F0704700127A00CC00002075
:10B4C00000F36F06000E270780D1F0080068890995
:10B4D000001C4E0E001BB70010B5032000F0C6F98B
:10B4E00000F0D5F9C4B204F0FB04204600F0E2F904
:10B4F00010BD10B5132000F0B9F900F0C8F9C4B2BE
:10B5000004F07F04204600F0D5F910BD10B503A06B
:10B5100001F07CFD01F0B9FB10BD00007761726E97
:10B52000696E67A3BB486172644661756C7420489C
:10B53000616E646C65720D0A0000000010B5012098
:10B5400000F094F900F0A3F9C4B244F001042046DD
:10B5500000F0B0F910BD10B500F006F810BD10B540
:10B5600000F002F810BD000008B5002000903C4833
:10B5700000793C4908703A48C0793B490870084650
:10B58000007800F00100002858D13648007800F01B
:10B590000400042863D13348007800F00200022838
:10B5A0001ED12F48007900F0010090B12C4840795D
:10B5B0002E4909682E4A126888542D480068401C9C
:10B5C0002B4908602648807840F00800244988709C
:10B5D00045E02348807820F02000214988703EE033
:10B5E0002048007800F0010008B31E48007800F001
:10B5F0004000402812D11F4800681F490968405C7C
:10B60000174948711C480068401C1B4908601448D1
:10B61000807820F020001249887020E0104840799E
:10B6200000909DF80000401CC0B2009017E00C484C
:10B63000807820F020000A49887010E0084880795E
:10B6400000F0C000401C064988710846807940F02F
:10B65000010088710846C07940F00100C87108BD3A
:10B6600000700140F0000020F100002000010020E7
:10B67000F4000020FC000020F800002030B530B9B4
:10B68000534C646A24F47F44514D6C621AE00128E3
:10B690000BD14F4C646A24F47F444D4D6C622C46B0
:10B6A000646A44F42A446C620CE002280AD1484CD3
:10B6B000646A24F47F44464D6C622C46646A44F408
:10B6C0007F446C6232B9424C246A24F44034404DC9
:10B6D0002C621AE0012A0BD13D4C246A24F4403438
:10B6E0003B4D2C622C46246A44F400342C620CE05E
:10B6F000022A0AD1364C246A24F44034344D2C6298
:10B700002C46246A44F440342C6233B9304C646AC9
:10B7100024F47F042E4D6C621AE0012B0BD12C4CCB
:10B72000646A24F47F042A4D6C622C46646A44F4F3
:10B730002A046C620CE0022B0AD1254C646A24F4C2
:10B740007F04234D6C622C46646A44F47F046C626F
:10B7500031B91F4C646A24F0FF041D4D6C6222E075
:10B7600001290FD11B4C1A4D80352C60184C646A8E
:10B7700024F0FF04164D6C622C46646A44F0AA045F
:10B780006C6210E002290ED1124C114D80352C60F4
:10B790000F4C646A24F0FF040D4D6C622C46646A01
:10B7A00044F0FF046C620A4C246844F00544084DE0
:10B7B0002C6000BF064C246804F00044B4F1004F34
:10B7C000F8D0034C246844F00104014D2C6030BDD6
:10B7D00000100540FFFF1F0010B500214FF0804012
:10B7E000FEF76CFE0121C807FEF768FE00214FF04E
:10B7F0000040FEF763FE10BD10B50246002001B9FF
:10B800000121052A2FD2DFE802F0030C20262A00AE
:10B810004FF04023DB6923F001034FF04024E36144
:10B8200022E04FF04023DB6943F001034FF0402456
:10B83000E3612346DB6823F00F03E3602346DB6804
:10B840000B43E3600123A3610EE04FF04023DB686C
:10B8500003F00F0008E04FF04023D86C04E04FF0F5
:10B860004023D96400E000BF00BF10BD10B50446FE
:10B8700000210C20FFF7FEFB002001F00FF920460D
:10B8800001F00CF901210C20FFF7F4FB10BD10B5FD
:10B89000002400210C20FFF7EDFBC02001F0FEF892
:10B8A000FF2001F0FBF8044601210C20FFF7E2FB2A
:10B8B000204610BD10B5044600210C20FFF7DAFB2E
:10B8C000802001F0EBF8204601F0E8F801210C207F
:10B8D000FFF7D0FB10BD70B50446082C06DA19201E
:10B8E000FFF7C4FF0020FFF7E5FF0CE02046E1175B
:10B8F00004EB5171C910491ECDB21920FFF7B6FFF4
:10B900002846FFF7D7FF70BD70B50446082C06DA4D
:10B910001820FFF7ABFF0020FFF7CCFF0CE020461C
:10B92000E11704EB5171C910491ECDB21820FFF781
:10B930009DFF2846FFF7BEFF70BD70B504460D465B
:10B94000082C1DDA1420FFF791FF0020FFF7B2FF4B
:10B950001520FFF78BFFE0B2FFF7ACFF681EC6B201
:10B960001A20FFF783FF3046FFF7A4FF681EC0F3DD
:10B9700007261B20FFF77AFF3046FFF79BFF2BE0DF
:10B980002046E11704EB5171C910491ECEB21420B4
:10B99000FFF76CFF3046FFF78DFF2046E11704EB01
:10B9A0005171C910A4EBC101CEB21520FFF75EFFA3
:10B9B0003046FFF77FFF681EC6B21A20FFF756FF1A
:10B9C0003046FFF777FF681EC0F307261B20FFF7FE
:10B9D0004DFF3046FFF76EFF70BD70B50446082C72
:10B9E0000CDA1620FFF742FF0020FFF763FF172055
:10B9F000FFF73CFFE0B2FFF75DFF1AE02046E117DA
:10BA000004EB5171C910491ECDB21620FFF72EFF6D
:10BA10002846FFF74FFF2046E11704EB5171C9108C
:10BA2000A4EBC101CDB21720FFF720FF2846FFF796
:10BA300041FF70BD70B505460C462846FFF716FF5E
:10BA40002046FFF737FF70BD10B5002401F07BF8EA
:10BA50000446204610BD70B50446601EC5B21F20C6
:10BA6000FFF704FF2846FFF725FF70BD70B50446B9
:10BA7000601EC5B21E20FFF7F9FE2846FFF71AFF29
:10BA800070BD70B50446601EC5B21C20FFF7EEFE07
:10BA90002846FFF70FFF1D20FFF7E8FE2812FFF7EB
:10BAA00009FF70BD2DE9F04106460F4614461D46BC
:10BAB000DDF818803946304601F038F9294620462D
:10BAC00001F018F901F05BF9FEF76FFEBDE8F081B7
:10BAD00010B50C48C07840F080000A49C87008468C
:10BAE000407920F0800048716420FEF789FF054806
:10BAF000407940F08000034948716420FEF780FFE0
:10BB000010BD00000090014010B56420FEF778FFE2
:10BB1000FFF7DEFF01F0F2F96420FEF771FF00BFCE
:10BB2000FFF792FF00F002000028F9D100F038F989
:10BB300010BD00002DE9FE4F0024464C4648B4FBE2
:10BB4000F0F100FB11404549B0FBF1F00290029882
:10BB5000052804D94048B4FBF0F0441C02E03E48FC
:10BB6000B4FBF0F43E490C7004EB84043D490C70C6
:10BB70003D490C7008460078642801DD6420087097
:10BB800038480078642802DD64203649087034485B
:10BB90000078412802DD4120314908704FF0030848
:10BBA000C146C2464FF0050B0521019100912D4879
:10BBB000007887002C4800788600294800788500A6
:10BBC0000520FFF753FE4FEA881141EA4B01C5F308
:10BBD000002241EA0200FFF76DFE0720FFF746FE54
:10BBE0004FEA8A12009942EA4101C7F3002241EA72
:10BBF0000200FFF75FFE0920FFF738FE4FEA8912C7
:10BC0000019942EA4101C6F3002241EA0200FFF72E
:10BC100051FE0620FFF72AFEE8B2FFF74BFE082090
:10BC2000FFF724FEF8B2FFF745FE0A20FFF71EFEDD
:10BC3000F0B2FFF73FFE0020FFF718FE0120FEF7ED
:10BC4000DFFE8020FFF736FE0120FEF7D9FEBDE8BB
:10BC5000FE8F00008013100240420F00A0860100FA
:10BC60002900002028000020270000202DE9F041B5
:10BC700005460C4616461F46DDF8188000F08AFF80
:10BC8000304601F00EF80CB900F093FF012C01D101
:10BC900000F09EFF022C01D100F0A9FF032C01D17E
:10BCA00000F0B4FF384601F016F8404601F004F801
:10BCB000012D01D101F056F80DB901F06AF8BDE887
:10BCC000F08170B505462921E020FFF7B3FE03217E
:10BCD000E120FFF7AFFE4FF47A7090FBF5F041F6EC
:10BCE000846191FBF0F084B2A01E84B2E1B2E22044
:10BCF000FFF7A0FE2112E320FFF79CFE0121E420C4
:10BD0000FFF798FEFEF763FD0120FEF779FE70BD98
:10BD10002DE9F04106460C4615461F46DDF8188011
:10BD2000102E01D1FFF74BFB182E01D1FFF729FB95
:10BD3000202E01D1FFF734FB012C01D1FFF74EFB80
:10BD4000022C01D1FFF759FB032C01D1FFF764FB53
:10BD5000042C01D1FFF76FFB012D01D1FFF7D5FABC
:10BD6000022D01D1FFF7E0FA032D01D1FFF7EBFA25
:10BD7000042D01D1FFF7F6FA0FB9FFF7ACFA012F46
:10BD800001D1FFF7B5FAB8F1000F01D1FEF752FE6D
:10BD9000B8F1010F01D1FFF791FABDE8F081000081
:10BDA00010B5FFF7C7FE03480078FFF78AFF00F0E1
:10BDB0003CFF10BD2800002010B501210C20FEF72B
:10BDC0007DFB10BD10B50446E1B22020FFF732FE26
:10BDD000C4F307212120FFF72DFEC4F307412220E1
:10BDE000FFF728FE210E2320FFF724FE10BD10B51B
:10BDF0000446E1B22420FFF71DFE21122520FFF7A3
:10BE000019FE10BD70B504460D46E1B22620FFF7BD
:10BE100011FE21122720FFF70DFEE9B22820FFF7BF
:10BE200009FE29122920FFF705FE70BD002100221E
:10BE300000BF11E00846002208E000F001031BB13A
:10BE4000074B83EA500000E04008521C082AF4D354
:10BE5000044B43F82100491CFF29EBD9704700002F
:10BE60002083B8ED0801002010B503A001F0CEF842
:10BE700000F00BFF10BD00007761726E696E67A362
:10BE8000BB4D656D4D616E6167652048616E646C88
:10BE900065720D0A0000000010B50220FFF7E6FCF5
:10BEA000FFF7F5FCC4B204F0FB0404F0FD042046E7
:10BEB000FFF700FD10BD10B50320FFF7D7FCFFF71B
:10BEC000E6FCC4B204F0FD0404F0FE042046FFF7D3
:10BED000F1FC10BD10B55E20FFF7C8FCFFF7D7FCE2
:10BEE000C4B204F0FB042046FFF7E4FC10BD0000E0
:10BEF00010B503A001F08AF800F0C7FE10BD0000E5
:10BF00007761726E696E67A3BB4E4D492048616EC2
:10BF1000646C65720D0A00002DE9F0410746884601
:10BF200014461D46284600F033F8C5F1030007FA11
:10BF300000F60720284100EA0800064306F007063D
:10BF4000E21704EBD2625211920002F1E022D2F821
:10BF500000212146E31704EBD3635B11A4EB431CE0
:10BF6000012303FA0CF31A432046E31704EBD363CF
:10BF70005B119B0003F1E023C3F800210348005D3F
:10BF800040EA461001490855BDE8F08100E400E0B0
:10BF90000146072323EA01021202054B18684FF6F7
:10BFA000FF031840034B18431043014B18607047C0
:10BFB0000CED00E00000FA054A0A52020243014B70
:10BFC0001A60704708ED00E010B57348446C04F047
:10BFD000010040B171A001F019F86F48406C40F0C9
:10BFE00001006D49486404F00200022808D170A0E5
:10BFF00001F00CF86848406C40F002006649486463
:10C0000004F01000102808D16EA000F0FFFF624875
:10C01000406C40F010006049486404F02000202883
:10C0200008D16DA000F0F2FF5B48406C40F02000AA
:10C030005949486404F48070B0F5807F13D15648A4
:10C04000806800F48010B0F5801F03D167A000F075
:10C05000DDFF02E06BA000F0D9FF4F48406C40F4D8
:10C0600080704D49486404F40070B0F5007F08D139
:10C070006AA000F0CBFF4848406C40F4007046498D
:10C08000486404F48060B0F5806F13D14248806842
:10C0900000F40010B0F5001F03D166A000F0B6FF59
:10C0A00002E06AA000F0B2FF3B48406C40F48060C0
:10C0B0003949486404F40060B0F5006F08D169A004
:10C0C00000F0A4FF3448406C40F4006032494864FA
:10C0D00004F48050B0F5805F13D12F48806800F4DD
:10C0E0008000B0F5800F03D164A000F08FFF02E064
:10C0F00068A000F08BFF2848406C40F4805026492F
:10C10000486404F40050B0F5005F08D167A000F067
:10C110007DFF2148406C40F400501F49486404F4FE
:10C120008040B0F5804F13D11B48806800F40000B8
:10C13000B0F5000F03D163A000F068FF02E067A034
:10C1400000F064FF1448406C40F480401249486499
:10C1500004F40040B0F5004F08D166A000F056FF8F
:10C160000D48406C40F400400B49486404F48030B2
:10C17000B0F5803F08D165A000F048FF0648406C4C
:10C1800040F48030044948640348006A6349084326
:10C190000149086210BD000000400340504349209F
:10C1A00056445F4C20746F756368210D0A000000CF
:10C1B0005043492056445F4820746F756368210DD1
:10C1C0000A0000005043492054445F4C20746F75AE
:10C1D0006368210D0A0000005043492054445F4821
:10C1E00020746F756368210D0A0000005344494FA5
:10C1F0002064796E616D69632D3020746F7563689A
:10C20000210D0A005344494F207374617469632DF2
:10C210003020746F756368210D0A00005344494F44
:10C22000207374617469632D3120746F75636821A4
:10C230000D0A00005344494F2064796E616D6963B3
:10C240002D3120746F756368210D0A005344494FE6
:10C25000207374617469632D3220746F7563682173
:10C260000D0A00005344494F207374617469632DB3
:10C270003320746F756368210D0A00005344494FE1
:10C280002064796E616D69632D3220746F75636807
:10C29000210D0A005344494F207374617469632D62
:10C2A0003420746F756368210D0A00005344494FB0
:10C2B000207374617469632D3520746F7563682110
:10C2C0000D0A00005344494F2064796E616D696323
:10C2D0002D3320746F756368210D0A005344494F54
:10C2E000207374617469632D3620746F75636821DF
:10C2F0000D0A00005344494F207374617469632D23
:10C300003720746F756368210D0A00006E767261C4
:10C310006D20636C65616E210D0A000000FFFF0057
:10C320000448006840F01F004FF04021C1F8900021
:10C33000704700009040004010B51220FFF796FAB9
:10C34000FFF7A5FAC4B244F080042046FFF7B2FA22
:10C3500010BD10B51220FFF789FAFFF798FAC4B2A2
:10C3600004F0F8042046FFF7A5FA10BD1349098828
:10C3700021F00101114A11801146098841F00401A0
:10C38000118001210E4A11800E4A11700E49097860
:10C390000E4A1170114609786C290DD0012004E075
:10C3A0000949095C094A1154401C09490988884215
:10C3B000F6DB0021064A1180704700000070004043
:10C3C000320000203400002018050020183B002017
:10C3D000300000200A48008840F004000849088026
:10C3E00008480078401C074908700846007805286E
:10C3F00004DB00200870012003490870704700002A
:10C4000000800040760000207400002000B500F09D
:10C410000DF800BD00B500F009F800BD00B500F052
:10C4200005F800BD00B500F001F800BD00201F496F
:10C4300008781E496C3991F8441001F0100141B19F
:10C440001A492839097841F01001184A6C3A82F8E3
:10C45000441016492639097801F0100139B1134901
:10C460002639097841F01002104926390A700F491F
:10C470002439097801F0100141B10C4924390978B7
:10C4800041F01001094A6C3A82F8481007492239F4
:10C49000097801F0100139B104492239097841F0D5
:10C4A0001002024922390A70704700006C80014076
:10C4B0002DE9F04705460E4614461F46DDE908897A
:10C4C0002DB1012D03D0022D01D0032D00D103E0A9
:10C4D000252197A000F0E6FF042C06D02CB1012CFA
:10C4E00003D0022C01D0032C00D103E0262190A020
:10C4F00000F0D8FF35B1012D47D0022D7DD0032D9E
:10C500007CD1CEE09148406940F001008F494861FC
:10C510008F48007A20F001008D4908720846406873
:10C5200020F0070048600846406804F0070108430F
:10C53000874948600E700846007A40F0080008728B
:10C540000846C0F81080C76081486E30007840F01F
:10C5500001017F486E300170401E007840F00101FB
:10C560007B486D300170401E007840F00100784932
:10C5700081F86C000846007A40EA89000872084693
:10C58000007A40F001000872CFE07048406940F046
:10C5900002006E4948616E48407A20F001016C4803
:10C5A0004172406820F07000694948600846406860
:10C5B00004F0070140EA0110654948600E70084622
:10C5C000407A40F0080162484172C0F81C808761DF
:10C5D0005F486E30007840F002015D486E300170B7
:10C5E000401E007840F0020159486D300170401E35
:10C5F000007840F00200564901E00FE094E081F835
:10C600006C000846407A40EA8900C1B25048417245
:10C61000407A40F001014E48417286E04B48406943
:10C6200040F00400494948614948807A20F00101FE
:10C6300047488172406820F4E060454948600846F8
:10C64000406804F0070140EA0120414948604E700B
:10C6500008213F488172C0F8288047623C486E300C
:10C66000007840F004013A486E300170401E0078B6
:10C6700040F0040136486D300170401E007840F0F3
:10C680000400334981F86C000846807A40EA89004A
:10C69000C1B22F488172807A40F001012C4881722A
:10C6A00043E02A48406940F004002849486128488E
:10C6B000C07A20F001012648C172406820F4E040B1
:10C6C000234948600846406804F0070140EA013009
:10C6D0001F4948604E7008211D48C172C0F834805F
:10C6E00007631B486E30007840F0080118486E3030
:10C6F0000170401E007840F0080115486D3001704F
:10C70000401E007840F00800114981F86C0008468E
:10C71000C07A40EA8900C1B20D48C172C07A40F0C7
:10C7200001010B48C17200E000BF00BFBDE8F08707
:10C730004D43555F6472765C6472765C7372635CC1
:10C7400070776D5F6472762E630000000010004009
:10C750000080014010B500F07DF910BD10B503A0B8
:10C7600000F054FC00F091FA10BD00007761726E89
:10C77000696E67A3BB50656E6453562048616E6452
:10C780006C65720D0A0000002DE9F04104460D466B
:10C7900017460026E000B0FBF5F0401CC0F3450052
:10C7A0000A498872A000B0FBF5F08609300A48708B
:10C7B0000E700846807840F02C00887002232022FA
:10C7C00001210846FFF7A8FBBDE8F08100300140D9
:10C7D000064840790548407900F01000102803D140
:10C7E00002498879487900BF704700000040014045
:10C7F00010B57348407900F0200020287BD17049A3
:10C8000088797049097899B9A5280BD16E490A78B9
:10C810000978491C6C4B19706C4988540121694A8C
:10C820001170CBE00021674A1170674A1170C5E0B2
:10C8300064490978012913D15A280BD162490A7831
:10C840000978491C604B19706049885402215D4A7F
:10C850001170B3E000215B4A11705B4A1170ADE0CA
:10C8600058490978022913D101280BD156490A7871
:10C870000978491C544B1970544988540321514A72
:10C8800011709BE000214F4A11704F4A117095E0E2
:10C890004C49097803290BD14B490A780978491C7E
:10C8A000494B1970494988540421464A117085E062
:10C8B0004449097804290BD143490A780978491C6D
:10C8C000414B19704149885405213E4A117075E069
:10C8D0003C49097805290FD13D4908700A783A4941
:10C8E0000B780978491C384C21703849CA54062104
:10C8F000344A117062E062E03249097806290BD1AE
:10C9000031490A780978491C2F4B19702F498854EE
:10C9100007212C4A117051E02A49097807290BD1C7
:10C9200029490A780978491C274B197027498854E6
:10C930000821244A117041E022490978082928D1A8
:10C9400023490978891E89B91F490A780978491C41
:10C950001D4B19701D49885400211D4A1170012179
:10C960001C4A11700021174A117027E016490A78F5
:10C970000978491C144B19701449885419460A78CF
:10C9800013490978891D8A4218D109210D4A11706D
:10C9900014E00C490978092910D10B490A78097863
:10C9A000491C094B1970094988540021084A117023
:10C9B0000121084A11700021024A117000BF10BD08
:10C9C00000D00140BD000020BC0000206E7B002094
:10C9D000BF000020010000202DE9F04104460D4673
:10C9E00017460026E000B0FBF5F0401CC0F3450000
:10C9F0000A498872A000B0FBF5F08609300A487039
:10CA00000E700846807840F02C00887002233D228A
:10CA100000210846FFF780FABDE8F08100D0014010
:10CA20001CB510208DF8010000208DF800008DF855
:10CA300005008DF804008DF8030007208DF8020032
:10CA400000208DF806006946014800F048F81CBD3A
:10CA5000000001401CB500208DF8000010208DF86A
:10CA6000010007208DF8020008208DF80300042043
:10CA70008DF8040000208DF805008DF80600694649
:10CA8000054800F02CF80121034800F01DF80121B1
:10CA90000C20FEF70FF91CBD00100140014600BF3D
:10CAA0000848C08A00F008000028F9D1054A9174AE
:10CAB00000BF0448C08A00F001000028F9D10148F5
:10CAC000807C70470010014021B1827842F0400222
:10CAD000827003E0827802F0BF028270704710B566
:10CAE00000224FF6FF73C38280238371C3714278A3
:10CAF00022F00F028B781A434270827800220B7961
:10CB0000CC7823438C7923434C7823431A43827097
:10CB10004B78102B0AD14B7903700023C3720E237C
:10CB20008372837B43F00803837303E00023C372A3
:10CB3000012383720023C370837843F04003837022
:10CB40000123C37210BD10B5002400210C20FEF794
:10CB500091FA4020FFF7A2FFFF20FFF79FFFC4B22A
:10CB600001210C20FEF786FA204610BD10B503A067
:10CB700000F04CFA00F089F810BD00007761726E89
:10CB8000696E67A3BB5356432048616E646C65723F
:10CB90000D0A000010B58520FEF768FEFEF777FE4F
:10CBA000C4B244F0080404F0FB042046FEF782FE01
:10CBB00010BD10B58520FEF759FEFEF768FEC4B221
:10CBC00004F07F0404F0BF042046FEF773FE10BD9E
:10CBD00010B58520FEF74AFEFEF759FEC4B204F0F8
:10CBE0007F0444F040042046FEF764FE10BD10B5FB
:10CBF0008520FEF73BFEFEF74AFEC4B244F08004F7
:10CC000004F0BF042046FEF755FE10BD10B5852088
:10CC1000FEF72CFEFEF73BFEC4B244F0800444F065
:10CC200040042046FEF746FE10BD10B5FEF786FC18
:10CC3000FFF732F9FEF750FCFFF73DF9FFF77CFBF9
:10CC400000F0C0F9FFF785FBFEF753FC00F0C7F9D1
:10CC5000FDF774FE4FF4F0714FF44870FEF76DFE6F
:10CC60008C20FEF7BAFEA020FEF74EFE1420FEF741
:10CC700032FE1420FEF705FF0C20FEF7F7FE03201E
:10CC8000FEF7E9FEFFF726F910BD10B5FDF743FDED
:10CC90004FF04020C06D40F008004FF04021C865C3
:10CCA00010BD10B50446601E84B28420FEF7DEFD80
:10CCB000E0B2FEF7FFFD10BD10B504468C20FEF774
:10CCC000D5FDE0B2FEF7F6FD8D20FEF7CFFD201278
:10CCD000FEF7F0FD10BD10B504468E20FEF7C6FD30
:10CCE000E0B2FEF7E7FD8F20FEF7C0FD2012FEF751
:10CCF000E1FD10BD70B504460D466C20FEF7B6FD93
:10CD0000E0B2FEF7D7FD6D20FEF7B0FD2012FEF772
:10CD1000D1FD6E20FEF7AAFDE8B2FEF7CBFD6F2035
:10CD2000FEF7A4FD2812FEF7C5FD70BD70B50446E0
:10CD30000D466820FEF79AFDE0B2FEF7BBFD6920C4
:10CD4000FEF794FD2012FEF7B5FD6A20FEF78EFD7A
:10CD5000E8B2FEF7AFFD6B20FEF788FD2812FEF764
:10CD6000A9FD70BD10B58620FEF780FDFEF78FFD92
:10CD7000C4B244F010042046FEF79CFD10BD10B56F
:10CD80007620FEF773FDE020FEF794FDFDF716FD1B
:10CD900010BD10B58620FEF769FDFEF778FDC4B220
:10CDA00004F0EF042046FEF785FD10BD704700003B
:10CDB0002DE9FF4704460D4617464FF00009344B56
:10CDC0000FCB8DE80F00C8460026032C01DC002C99
:10CDD00010DAFEF73FFB2F49086000210220FEF722
:10CDE0000BFD401C2B490968B1FBF0F02A49086093
:10CDF000BDE8FF87FEF72EFB804628480460032C21
:10CE000001D105B901255DF82410681CB1FBF0F6CD
:10CE10002348864205D146450ED00320FDF759FC34
:10CE20000AE02048804505D8864203D90120FDF755
:10CE300050FC01E04FF001092046FDF76DFA29464C
:10CE40000120FDF793FB39460120FEF7D5FCFEF7E4
:10CE500001FB1049086000210220FEF7CDFC401CB8
:10CE60000C490968B1FBF0F00B49086009480068FB
:10CE70000C49884203D81020FDF72BFC05E0B9F1DE
:10CE8000000F02D00120FDF724FC00BFB0E7000036
:10CE900034DC0008C4000020C8000020CC000020C2
:10CEA00080D1F0080087930310B50A4800F02EFBEC
:10CEB000012200210220FFF77BFF00231A460121F7
:10CEC0001846FDF78DFC00231A4601211846FEF78F
:10CED000D5FB10BD90D003000648006840F47000F8
:10CEE0000449086004486FF308000249803908606B
:10CEF0007047000088ED00E000A0000870B5002435
:10CF00000026002500BFFEF79FFD00F00200F8B9E3
:10CF10000120FDF775FD0120FEF7A8FC0120FDF7BB
:10CF20006FFDFEF7B4FCC6B206F08000802802D187
:10CF3000012500240FE00120FDF762FD0120FEF72E
:10CF400095FC0120FDF75CFD8020FEF7B3FC02E0BC
:10CF50000025601CC4B225B9052C02D1FEF7B8FD2E
:10CF60000024002DCFD070BD00B500F001F800BD49
:10CF70000648008840F008000449088000BF0348C4
:10CF8000008800F080000028F9D170470060004060
:10CF90007047000010B503A000F038F8FFF775FEE9
:10CFA00010BD00007761726E696E67A3BB55736137
:10CFB00067654661756C742048616E646C65720DBE
:10CFC0000A00000010B51220FEF750FCFEF75FFCCF
:10CFD000C4B204F0F7042046FEF76CFC10BD10B597
:10CFE0001320FEF743FCFEF752FCC4B204F0BF046A
:10CFF0002046FEF75FFC10BD45F255500249C8803F
:10D000004000C88070470000005000400FB4054B3E
:10D0100010B503A9044A029800F018F810BC5DF896
:10D0200014FB0000F5D500080401002002E008C848
:10D03000121F08C1002AFAD170477047002001E092
:10D0400001C1121F002AFBD1704700002DE9FF4FDC
:10D050008DB00F460546002606E025280BD0DDE9F9
:10D060000F1290476D1C761C28780028F5D111B05E
:10D070003046BDE8F08F0024A246A1460122E949CE
:10D0800000E0044315F8013F203B02FA03F0084298
:10D09000F7D128782A2810D06FF02F022878A0F135
:10D0A0003001092914D80AEB8A0102EB410144F04E
:10D0B000020400EB010A6D1CF0E701CF5FEA000AF1
:10D0C00003D544F40054CAF1000A44F002046D1C74
:10D0D00028782E2817D115F8010F44F004042A28C7
:10D0E0000ED06FF02F022878A0F1300109290AD85C
:10D0F00009EB890102EB410100EB01096D1CF2E72C
:10D1000057F8049B6D1C28786C280FD006DC4C283F
:10D1100017D068280DD06A2814D104E0742810D0E4
:10D120007A280FD10DE044F400140AE044F480148E
:10D1300001E044F440146978814202D104F580147E
:10D140006D1C6D1C28786E281ED00CDC632830D036
:10D1500004DC00288BD0582811D19FE0642867D0C8
:10D1600069280CD164E073282DD004DC6F2872D0BC
:10D17000702804D194E075286ED078286DD0DDE950
:10D180000F129047761C4BE1C4F30250022806D0E0
:10D19000032809D0042801CF09D0066040E101CF5F
:10D1A000F117C0E900613BE101CF068038E106706C
:10D1B00036E117F8040B8DF8000000208DF801000F
:10D1C000EB46012003E057F804BB4FF0FF30610746
:10D1D0004FF0000102D40DE008F1010188464945F5
:10D1E0000FDA8045F8DB1BF808100029F4D108E0BD
:10D1F00008F1010188468142FADB1BF8081000297A
:10D20000F6D1DDE90F23AAEB08008146214600F0A4
:10D2100031F9304400EB080604E0DDE90F121BF899
:10D22000010B9047B8F10108F7D221464846F2E0D9
:10D230000A21C4F302524FF0000B0891022A04D0D5
:10D2400001CFC117032A09D00AE0FF1D27F0070705
:10D25000F7E8020108E02CE01EE01FE000B2C11771
:10D26000042A01D140B2C117021E71F1000206DA90
:10D270000023D0EB030063EB01012D2202E0220525
:10D2800004D52B228DF82420012203E0E20701D0EF
:10D290002022F7E7904653E00A210BE0102109E035
:10D2A00010214FF0000B44F004044FF008090891DE
:10D2B00003E008214FF0000B0891C4F30252022A48
:10D2C00004D001CF0021032A06D006E0FF1D27F07D
:10D2D0000707F7E8020103E080B2042A00D1C0B2D8
:10D2E0004FF0000822072BD52A78702A07D0DDF8E6
:10D2F00020C08CF0100C5CEA0B0C05D00EE0402234
:10D300008DF82420012208E050EA010306D03023E2
:10D310008DF824308DF8252002229046089B83F05A
:10D32000080353EA0B030BD150EA010201D1620753
:10D3300006D530228DF824204FF00108A9F101090B
:10D340002A78582A04D038A20B9208AA0A920BE035
:10D350003AA2F9E75B46089AFCF73EFF0B9B9B5C01
:10D360000A9A521E0A92137050EA0102F2D10A98E8
:10D37000ADEB000000F1200B600702D524F48034EF
:10D3800001E04FF00109D94502DDA9EB0B0000E0F7
:10D39000002000EB0B0141440890AAEB010AE003D6
:10D3A00006D4DDE90F232146504600F063F8064419
:10D3B0004FF0000908E009A911F80900DDE90F1292
:10D3C000904709F10109761CC145F4DBE0030CD557
:10D3D000DDE90F232146504600F04CF8064404E0F6
:10D3E000DDE90F1230209047761C0899481E0890FE
:10D3F0000029F5DC08E00A980A990078491C0A918E
:10D40000DDE90F129047761CBBF10001ABF1010B77
:10D41000F1DC21465046DDE90F2300F019F80644FF
:10D420006D1C21E60928010030313233343536379E
:10D430003839616263646566000000003031323360
:10D440003435363738394142434445460000000000
:10D450002DE9F041044600251E461746880404D4F1
:10D4600005E039462020B0476D1C641EF9D52846DA
:10D47000BDE8F0812DE9F041044600251E469046A6
:10D48000C80301D5302700E02027880404D505E033
:10D4900041463846B0476D1C641EF9D52846BDE8A4
:10D4A000F081000004460D462A46214602A0FFF7FF
:10D4B000ADFD00BFFEE7000057726F6E6720706120
:10D4C00072616D65746572732076616C75653A2062
:10D4D00066696C65202573206F6E206C696E65200F
:10D4E00025640D0A000000004FF04021896821F0FA
:10D4F000FF014FF04022916011468968014391601D
:10D500001146896941F002019161704701B500BF80
:10D510000098411E00910028FAD108BD1CB50446B0
:10D520000020022104231A46CDE900100120FEF755
:10D53000BFFFFFF70FF9FEF7E7FA2C48C07840F07D
:10D5400040002A49C8700846407940F040004871C0
:10D55000012027490870FFF763FA0020FEF732FC2C
:10D560004FF44870FEF743FC00210846FEF74AFCE2
:10D570000020FDF7FAF84FF44870FDF70BF9002191
:10D580000846FCF79FFE4FF4F0714FF44870FCF72B
:10D5900085FE5CB14FF6FF7040F2DF1340F21F32A0
:10D5A000002100900846FEF77DFA0AE040F21F5085
:10D5B00040F2DF1340F21F32002100900846FEF7D0
:10D5C00071FA002003460122114600901820FEF750
:10D5D0009FFB4FF4C87043000522002100900120FA
:10D5E000FEF744FBFDF733FA1CBD0000009001403C
:10D5F0002600002000BF044A527902F04002002AAF
:10D60000F9D0014B987170470030014030B50246A7
:10D61000A523164804780078401C144D2870135533
:10D620005A23284604780078401C2870135501239B
:10D63000284604780078401C287013552846037843
:10D640000078401C2C462070D154032320460478D7
:10D650000078401C28701355002328460478007871
:10D66000401C287013552846007830BDBA000020B1
:10D6700030B50246A523204804780078401C1E4D92
:10D68000287013555A23284604780078401C2870C7
:10D6900013550123284604780078401C2870135540
:10D6A000284604780078401C28701355212328460A
:10D6B00004780078401C287013550223284604780B
:10D6C0000078401C287013550323284604780078FE
:10D6D000401C287013550123284604780078401C0C
:10D6E000287013552823284604780078401C287099
:10D6F00013552846007830BDBA0000200021E648C6
:10D70000FEF75AFCFFF7D0FB62B600224FF461210E
:10D71000E2480068FFF738F800224FF41641DF486E
:10D720000068FFF759F9DE48DE490860FEF77EFB26
:10D73000DB48DC490860DCA0FFF768FC0020FFF74D
:10D74000EDFEDFA2E1A1E4A0FFF760FCA2E1FFF79C
:10D7500053FCE84800780128F8D1E7480078401EDB
:10D7600081B2E648FCF7EBFF04462246E248017826
:10D77000E3A0FFF74BFCE0480078401E81B2DF4891
:10D78000FCF7DDFFDC490978491EDC4A515C884220
:10D7900010D0D9480078401E81B21046FCF7CFFF68
:10D7A0000446D5480078401ED4490A5C2146D9A0D9
:10D7B000FFF72CFCD1480078A5280AD0CF48407844
:10D7C0005A2806D0CD488078012802D0D6A0FFF78D
:10D7D0001DFC002406E0C948015DD7A0FFF716FC38
:10D7E000601CC4B2C44800788442F4DBC0A0FFF7D8
:10D7F0000DFCC248007920283CD1C048807901281E
:10D8000038D1BE48C079012834D1BC48C078CB4952
:10D81000087008460178CA48FFF7F8FE044621461A
:10D82000C748FCF78CFFC6490855601CC4B20020ED
:10D83000C4490870B0490870AE4908702146C04814
:10D8400000F0C8F91E20FDF7DBF8BC480178BC48A1
:10D85000FFF70EFF05460020BA490870A649087078
:10D86000A4490870B8A0FFF7D1FB2946B44800F0DE
:10D87000B1F90FE1A148007920285CD19F48807957
:10D88000022858D19D48C079012854D19B48407A3C
:10D890009A49097A4FF4807313FB0102AE4801885C
:10D8A000AEA0FFF7B3FB9548407A9449097A4FF44C
:10D8B000807212FB0100A849098888421AD1AAA0E7
:10D8C000FFF7A4FB002508E08C4A05F10B00115C72
:10D8D00099A0FFF79BFB681CC5B28848807AA842D4
:10D8E000F2DC83A0FFF792FB9B480088401C9A491A
:10D8F000088002E09EA0FFF789FB8048C0788F492E
:10D900000870084601788E48FFF780FE04462146DD
:10D910008B48FCF714FF8A490855601CC4B20020EC
:10D920008849087074490870724908702146844813
:10D9300000F050F9AEE07148007920282FD16F48EF
:10D94000807901282BD16D48C079022827D18CA07D
:10D95000FFF75CFB6948C078784908700846017891
:10D960007748FFF753FE044621467548FCF7E7FE6B
:10D9700073490855601CC4B20020724908705E49A2
:10D9800008705C490870744908800846018880A0C6
:10D99000FFF73CFB21466A4800F01CF97AE0574843
:10D9A0000079202828D155488079012824D153486E
:10D9B000C079022820D17AA0FFF728FB4F48C07811
:10D9C0005E490870084601785D48FFF71FFE04466F
:10D9D00021465B48FCF7B3FE59490855601CC4B2A8
:10D9E000002058490870444908704249087021468F
:10D9F000534800F0EFF84DE040480079202828D146
:10DA00003E488079012824D13C48C079022820D1A1
:10DA100068A0FFF7FBFA3948C07848490870084603
:10DA200001784748FFF7F2FD044621464448FCF7D9
:10DA300086FE43490855601CC4B200204149087065
:10DA40002D4908702B49087021463D4800F0C2F866
:10DA500020E05CA0FFF7DAFA2848C0783749087060
:10DA6000084601783648FFF7D1FD04462146344880
:10DA7000FCF765FE32490855601CC4B200203149EC
:10DA800008701D4908701B49087021462C4800F099
:10DA9000A1F800BF5BE6000000A00008C80000205D
:10DAA000000001080C0000202A2A2A626F6F746CA3
:10DAB0006F616465723121212A2A0D0A000000007D
:10DAC00031363A32313A3135000000004D6179206B
:10DAD00033302032303235002064617465203D20BF
:10DAE00025732C74696D65203D202573202020202E
:10DAF0000D0A000001000020BC0000206E7B002009
:10DB00007265763A256420636865636B3A25780D03
:10DB10000A000000257820636865636B5F65727298
:10DB20006F2025780D0A0000696C6C6567616C5F79
:10DB30006E6577210D0A000020257800BB000020CB
:10DB40005A7B0020BA0000207374617274207570D3
:10DB5000646174610D0A0000C00000202A2A2A2591
:10DB6000642025640D0A000062696E3A000000001E
:10DB70002A2A2A726570656174210D0A000000006E
:10DB80004F54412D66696E6973680D0A00000000EC
:10DB90006F74615F7365713D25640D0A00000000BC
:10DBA0004F54412D726571756573742D6661696C92
:10DBB0000D0A00004F54412D74696D656F75740D29
:10DBC0000A0000006F74686572206E6577210D0A87
:10DBD0000000000070B504460D4611A0FFF716FACC
:10DBE000002605E0A15D10A0FFF710FA701CC6B278
:10DBF000AE42F7DB0DA0FFF709FA00200BE000BFF3
:10DC00000B49497901F040010029F9D0215C084A0B
:10DC10009171411CC8B2A842F1DB002070BD000028
:10DC200061636B3A00000000202578000D0A0000B7
:10DC300000D0014000F36F06000E270780D1F008E6
:10DC40000068890964DC0008000000200801000069
:10DC50002CD000086CDD00080801002068CB000013
:10DC60003CD00008000000000000000000000000A0
:10DC700000000000000000000000000000000000A4
:10DC80000000000000000000000001000000000093
:10DC90000000000000000000000000000000000084
:10DCA0000000000000000000000000000000000074
:10DCB0000000000000000000000000000000000064
:10DCC0000000000000000000000000000000000054
:10DCD0000000000000000000000000000000000044
:10DCE000000000000060044058600440B060044040
:10DCF000086104400070044058700440B070044053
:10DD000008710440C0620440C0720440000000007A
:10DD10000000000000000000000000000000000003
:10DD200000000000000000000000000000000000F3
:10DD3000030000000060044058600440B0600440EC
:10DD400008610440C06204400000000000000000C0
:10DD50000000000000FF00000000000000000000C4
:0CDD6000000000000000000000000000B7
:040000050800A1410D
:00000001FF
